:100000000200128F999000037401F0900003E070D9
:10001000FA22787FE4F6D8FD75812202095FAE07E7
:10002000020003020B2B90020874FFF07E017F0791
:10003000A3EEF0A3EFF090020C74FFF0A3EEF0A398
:10004000EFF09002077401F090020BF0FB7A027956
:1000500007FF12006EE4FBFD7F011200E1E4FBFDEF
:050060007F01020BCE40
:10006B00020A4C43BA80EF6401706790FA32F09049
:10007B00FA3AF090000112055D90FA33F09000020D
:10008B0012058AFF90FA35E5F0F0A3EFF09000052A
:10009B0012055D90FA3BF090000612058AFF90FA6C
:1000AB003DE5F0F0A3EFF0120544640190FA3170D6
:1000BB0006E04480F08004E0547FF09000041205C9
:1000CB005D640190FA397006E04480F08004E054DE
:1000DB007FF053BA7F2243BA8090FA30E054F0F0AD
:1000EB00EDD3940374809480500BE0FEED25E02556
:1000FB00E0FDEE4DF0EBD3940374809480500690AA
:10010B00FA30E04BF0EF640190FA307006E0448077
:0D011B00F08004E0547FF053BA7F7F002293
:02012B0021DDD4
:0201330021DDCC
:02013B0021DDC4
:0201430021DDBC
:02014B0021DDB4
:0201530021DDAC
:02015B0021DDA4
:020163008078A2
:02016B008070A2
:020173008068A2
:02017B008060A2
:020183008058A2
:02018B008050A2
:020193008048A2
:02019B008040A2
:0201A3008038A2
:0201AB008030A2
:0201B3008028A2
:0201BB008020A2
:0201C3008018A2
:0201CB008010A2
:0201D3008008A2
:1001DB008000016BE508240AF582E43402F583E024
:1001EB0005082290020730070390020AE475F0011C
:1001FB001207690205442000E97F2ED2008018EF18
:10020B00540F2490D43440D4FF30040BEF24BFB4EC
:10021B001A0050032461FFE50960021509050CE57E
:10022B000C7002050B30070E900207E475F00112FB
:10023B000769EF02072102001E7403D2078003E453
:10024B00C207F508900207120780E4F509F50BF5D4
:10025B000CE50960077F2012022280F5750AFFC2A8
:10026B0001C200C202C203C205C206C2081201EEDD
:10027B00FF700D3007057F00120233AF0CAE0B225F
:10028B00B4255FC2D5C2041201EEFF24D0B40A001C
:10029B00501A75F00A780930D50508B6FF0106C665
:1002AB00A426F620D5047002D20380D924CFB41A29
:1002BB0000EF5004C2E5D204020434D20180C6D24E
:1002CB000080C0D20280BCD2D580BAD20580B47F68
:1002DB00201202222002077401B5090040F112011D
:1002EB00DFFF12022202025CD208D20680951201B5
:1002FB00DFFB1201DFFA1201DFF94A4B70067905B9
:10030B007A057BFF20022EE509602A7E008E82751E
:10031B00830012055D60060EEE650A70F0C2D5EB28
:10032B00C0E0EAC0E0E9C0E0EE12047BD0E0F9D017
:10033B00E0FAD0E0FB120544FF60AAEBC0E0EAC094
:10034B00E0E9C0E0120222D0E02401F9D0E0340051
:10035B00FAD0E0FBE50A0460DCD50AD980877BFF85
:10036B007A047977D202809C791080027908C206D0
:10037B00C2088008D2D5790A8004790AC2D5E50A69
:10038B00047002F50AE4FAFDFEFF1201DFFC7B08A4
:10039B002001131201DFFD7B1030000A1201DFFE7A
:1003AB001201DFFF7B20EC3382D592D55013C3E4CF
:1003BB003000069FFFE49EFEE42001039DFDE49CBC
:1003CB00FCE4CBF8C201EC700CCFCECDCCE824F81A
:1003DB00F870F38017C3EF33FFEE33FEED33FDEC14
:1003EB0033FCEB33FB994002FB0FD8E9EB300105F3
:1003FB00F8D0E0C448B201C0E00AEC4D4E4F782073
:10040B007B0070C2EAB50A0040BCC0E012047DD08C
:10041B00F0D0E0200104C4C0E0C4B201C0F012026D
:10042B000BD0F0D5F0EB02025C12078902F95303F3
:10043B00735802CA4C02C64203774F037F44037FB3
:10044B004902DF4303855503694603694503694741
:10045B0005255002CE2D02D22E02F52B02D62302F9
:10046B00F320050E2A028E48000002ED3F3F3F00AD
:10047B00790AA2D5200314300509B910020404B976
:10048B00080104A2D5200602500104200268920242
:10049B00B509005034C0E07F203003197F30A20231
:1004AB0072067205500F1204D4C202C206C205C2F4
:1004BB00087F30800F300503E9C0E01202223005BF
:1004CB0003D0E0F9D0E0B509CC3005177F30B91077
:1004DB000C1202227F583004077F788003B908037F
:1004EB001202223002057F2D0202227F202008F803
:1004FB007F2B2006F322920280CF286E756C6C291D
:10050B0000D2011201DF3001F8C201780930D501A8
:10051B0008F602028E2D504349581201DF2403B412
:10052B0005004001E490052093120213743A120265
:10053B0013D203750904020373BB010689828A83F4
:10054B00E0225002E722BBFE02E32289828A83E487
:10055B009322BB010CE58229F582E5833AF583E012
:10056B00225006E92582F8E622BBFE06E92582F831
:10057B00E222E58229F582E5833AF583E49322BBF7
:10058B000110E58229F582E5833AF583E0F5F0A3C6
:10059B00E0225009E92582F886F008E622BBFE0A24
:1005AB00E92582F8E2F5F008E222E5832AF583E9F2
:1005BB0093F5F0A3E9932275F008758200EF2FFFF6
:1005CB00EE33FECD33CDCC33CCC58233C5829BED20
:1005DB009AEC99E58298400CF582EE9BFEED9AFD24
:1005EB00EC99FC0FD5F0D6E4CEFBE4CDFAE4CCF9D4
:1005FB00A88222B800C1B90059BA002DEC8BF08447
:10060B00CFCECDFCE5F0CBF97818EF2FFFEE33FE14
:10061B00ED33FDEC33FCEB33FB10D703994004EBCC
:10062B0099FB0FD8E5E4F9FA227818EF2FFFEE3398
:10063B00FEED33FDEC33FCC933C910D7059BE99AAA
:10064B004007EC9BFCE99AF90FD8E0E4C9FAE4CC3B
:10065B00FB2275F010EF2FFFEE33FEED33FDCC33A5
:10066B00CCC833C810D7079BEC9AE899400AED9B8E
:10067B00FDEC9AFCE899F80FD5F0DAE4CDFBE4CC6D
:10068B00FAE4C8F922EB9FF5F0EA9E42F0E99D42AD
:10069B00F0E89C45F022E8600FECC313FCED13FD72
:1006AB00EE13FEEF13FFD8F122BB010DE58229F506
:1006BB0082E5833AF5830207405007E92582F80269
:1006CB000733BBFE07E92582F802074CE58229F5C3
:1006DB0082E5833AF583020759ECF0A3EDF0A3EE24
:1006EB00F0A3EFF022A8828583F0D083D08212078B
:1006FB0007120707120707120707E473E493A3C552
:10070B0083C5F0C583C8C582C8F0A3C583C5F0C532
:10071B0083C8C582C822BB010689828A83F0225016
:10072B0002F722BBFE01F322E6FB08E6F908E6FA24
:10073B0008E6CBF822E0F8A3E0F9A3E0FAA3E0FB8C
:10074B0022E2FB08E2F908E2FA08E2CBF822E49392
:10075B00F8740193F9740293FA740393FB22F8E093
:10076B00FBA3A3E0F925F0F0E58215827002158357
:10077B00E0FA38F022EBF0A3EAF0A3E9F022D08301
:10078B00D082F8E4937012740193700DA3A393F8C5
:10079B00740193F5828883E4737402936860EFA30A
:1007AB00A3A380DF900210EBF0A3EAF0A3E9F0EF34
:1007BB006401600302095C90000004F0E4A3F0A361
:1007CB00F0A3F0A3F0A3F0A3F0FFEFC39480748029
:1007DB009480500F74872FF582E43400F583E4F096
:1007EB000F80E7E4FFEFC3948074809480500F7404
:1007FB00072FF582E43400F583E4F00F80E79002D5
:10080B0010E0FBA3E0FAA3E0F9120544FFE59854CE
:10081B003F4FF598EF64C06008EF64406003020936
:10082B00019000021206B47F007E607D547C0012A2
:10083B0005FE9002131206E4E4FFFE7D01FC90021C
:10084B0013E0F8A3E0F9A3E0FAA3E0FBC3120690D0
:10085B0040037FFF22900213E0F8A3E0F9A3E0FA34
:10086B00A3E0FBC3E49BFFE49AFE740199FDE498BB
:10087B00FC9002131206E4900210E0FBA3E0FAA333
:10088B00E0F990000112055D64027032538EEF4364
:10089B008E01538EF7438E04900213E0FCA3E0FD10
:1008AB00A3E0FEA3E0FF78081206A18FD6900213F7
:1008BB00A3A3A3E0F5D753AFFB438E108077C28E73
:1008CB00538EFE5389BF5389CF438E40900213E062
:1008DB00FCA3E0FDA3E0FEA3E0FF78081206A18FC6
:1008EB008D900213A3A3A3E0F58BC2AB5389BF5327
:1008FB008FFDD28E803F900210E0FBA3E0FAA3E0C5
:10090B00F9120544FF7E00701490000812055D6417
:10091B00017005438E20801D538EDF8018EF64809D
:10092B004E701290000812055D64017005438780BC
:10093B00800353877F900210E0FBA3E0FAA3E0F95A
:10094B0090000712055D7004C29C8002D29C7F0050
:10095B00227FFF22120C3D120C15120026D2AF7B08
:10096B00FF7A0C794412024AC20CC209C20EC20AA7
:10097B00C20FC20BC210C20DE4FFFE74072FF5822B
:10098B0074013EF583EFF00FBF00010EE4B507EBEA
:10099B00EEB401E743BA8090FA31E04440F053BA29
:1009AB007F43BA8090FA39E04420F053BA7F300C81
:1009BB002130091EC20CC20943BA8090FA31E044BF
:1009CB0040F053BA7F43BA8090FA39E04420F05399
:1009DB00BA7F300E21300A1EC20EC20A43BA809073
:1009EB00FA41E04440F053BA7F43BA8090FA49E0B1
:1009FB004420F053BA7F300F21300B1EC20FC20BB5
:100A0B0043BA8090FA51E04440F053BA7F43BA8026
:100A1B0090FA59E04420F053BA7F301091300D8E8C
:100A2B00C210C20D43BA8090FA61E04440F053BA51
:100A3B007F43BA8090FA69E04420F053BA7F0209F1
:100A4B00B9C0E0C083C082C0D075D000C007AFBAB8
:100A5B0043BA8090FA32E030E006E054FEF0D20C5C
:100A6B0090FA32E030E204E054FBF090FA3AE030D6
:100A7B00E006E054FEF0D20990FA3AE030E104E0EF
:100A8B0054FDF090FA42E030E006E054FEF0D20E56
:100A9B0090FA42E030E204E054FBF090FA4AE03086
:100AAB00E006E054FEF0D20A90FA4AE030E104E0AE
:100ABB0054FDF090FA52E030E006E054FEF0D20F15
:100ACB0090FA52E030E204E054FBF090FA5AE03036
:100ADB00E006E054FEF0D20B90FA5AE030E104E06D
:100AEB0054FDF090FA62E030E006E054FEF0D210D4
:100AFB0090FA62E030E204E054FBF090FA6AE030E6
:100B0B00E006E054FEF0D20D90FA6AE030E104E02A
:100B1B0054FDF08FBAD007D0D0D082D083D0E03242
:100B2B00C0E0C083C082C0D075D000C00730983100
:100B3B00C298900006E07029900004E0C394807482
:100B4B008094804002E4F0900004E0FF04F074070E
:100B5B002FF582E43400F583E599F09000057405D8
:100B6B00F0309907C299900003E4F0D007D0D0D0B1
:100B7B0082D083D0E032EFFBD39401748094805009
:100B8B0009EB7004C2AC8002D2ACEDFF7E00D394B3
:100B9B0003748094805029EF700553B7EFC2BCEFFC
:100BAB0064014E700553B7EFD2BCEF64024E700573
:100BBB0043B710C2BCEF64034E700543B710D2BCF1
:100BCB007F002243BA8090FA38E054F0F0EDD394D2
:100BDB000374809480500BE0FEED25E025E0FDEEE4
:100BEB004DF0EBD3940374809480500690FA38E068
:100BFB004BF0EF640190FA387006E04480F080040B
:100C0B00E0547FF053BA7F7F00229002077440F0CC
:100C1B00A37402F0A31206F00001C20090020E743E
:100C2B0001F0FB7A027907FF1207AF7D017F01020A
:100C3B000B8153B1FC53B2FC225354433841384B14
:100C4B0036344434205541525420424D4D20546586
:100C5B0073742050726F6772616D6D65210D0A00A0
:00000001FF
